:020000040800F2
:1000000040160020D9010008350300083503000818
:1000100035030008350300083503000835030008E0
:10002000350300083503000835030008DF02000827
:10003000350300083503000835030008870200086F
:1000400035030008350300083503000835030008B0
:1000500035030008350300083503000835030008A0
:100060003503000835030008350300083503000890
:100070003503000835030008350300083503000880
:100080003503000835030008350300083503000870
:100090003503000835030008350300083503000860
:1000A0003503000835030008350300083503000850
:1000B000ED240008F11D0008511E0008350300085A
:1000C0003503000835030008350300083503000830
:1000D00035030008E5200008F52000083503000876
:1000E0003503000835030008350300083503000810
:1000F0003503000800F002F800F05AF80AA090E872
:10010000000C82448344AAF10107DA4501D100F0D2
:100110004FF8AFF2090EBAE80F0013F0010F18BF45
:10012000FB1A43F00103184780310000A0310000A2
:100130000A444FF0000C10F8013B13F0070408BF0D
:1001400010F8014B1D1108BF10F8015B641E05D0AB
:1001500010F8016B641E01F8016BF9D113F0080F60
:100160001EBF10F8014BAD1C0C1B09D16D1E58BFF2
:1001700001F801CBFAD505E014F8016B01F8016B29
:100180006D1EF9D59142D6D370470000002300249C
:1001900000250026103A28BF78C1FBD8520728BF97
:1001A00030C148BF0B6070471FB51FBD10B510BDF3
:1001B000DFF80CD0FFF7F8FF02F035FD02F0B0FFDA
:1001C000400E002003B4FFF7F1FF03BC02F0AEFFC6
:1001D00002F0E4B87047000072B6094880F309885D
:1001E000022080F31488BFF36F8FFFF7F1FF0548FB
:1001F0000047704704480549054A064B7047000010
:10020000400E0020F5000008400E0020400E0020A7
:1002100040120020400A00202DE9F04FC1F80CD018
:10022000D0F80CD0BDE8F08F002383F31188284666
:10023000A04701F06AF900F0D2FF00DF202080F330
:1002400011883648006810F4006F02BF002080F368
:1002500011887047EFF30980203880F309884FF048
:100260008071C1612E498A690968D37F8968926863
:1002700013B1914202D803E0914201D3294900E031
:1002800029498161704710B5202484F3118801F059
:1002900012F8002080F3118884F311881F4909683F
:1002A00011F4006F04BF80F3118810BDEFF30980D3
:1002B000203880F309884FF08071C16118498A693C
:1002C0000968D37F8968926813B1914202D803E02C
:1002D000914201D3134900E01349816110BDEFF34E
:1002E0000980203080F30988002080F3118870474E
:1002F0000E4910B500200860091D0D480860102146
:10030000072000F053F84FF400710A2000F04EF877
:100310008021BDE810400B2000F048B804ED00E05B
:10032000D0010020370200083B02000808ED00E081
:100330000003FA05FEE70000254B20F0030C10B483
:1003400063448207D3F800C0D20EFF2494402CEA05
:10035000040C91404CEA0101196000F01F020121D8
:10036000914042094FF0E02000EB8200C0F880127B
:10037000C0F8001110BC70478107C90E00F01F02C1
:10038000012303FA02F243094FF0E02C0CEB830344
:10039000C3F8802120F003020D4810440268FF23B7
:1003A00003FA01F122EA010101607047820720F09F
:1003B00003030848D20E184403684FF0FF0C0CFAF0
:1003C00002FC23EA0C0391401943016070470000CE
:1003D00000E400E018ED00E0202181F31188817F26
:1003E000491C8177002181F311887047202181F316
:1003F0001188817F4FF00002491E11F0FF018177C3
:1004000082F3118806BF017F0E297047417F01F0FA
:10041000030101290DD0022918BF7047D0E9041249
:100420001161D0E904124A61426C0146104600F0A5
:10043000CABAD0E904121161D0E904124A6100F08D
:100440002EBAF8B51D4616460F46069C00F0E7F991
:10045000002808BFF8BD202181F311882B463246C1
:100460003946009400F07CFF0446012060770021AB
:10047000204600F020FE002080F311882046F8BDC1
:10048000F8B51C4616460F46054600F0C8FA002887
:1004900008BFF8BD202181F31188009433463A4605
:1004A000696800F05DFF0446022060770021204665
:1004B000656400F000FE002080F311882046F8BD3E
:1004C000202383F3118803680B600160C9488069A9
:1004D000C1E90102002080F31188C860704702461C
:1004E000202383F311880368834209D013688B4269
:1004F00002D10868106003E01A461B688342F5D1F8
:10050000002080F311887047202181F31188B949B8
:100510008B69996B01EA000221EA000098630020D0
:1005200080F3118810467047202181F31188B1496A
:1005300089698A6B10438863002181F311887047B1
:1005400010B5826B11438163027F082A0DD0092AFE
:1005500018BF10BD426A32EA010118BF10BD00BFCA
:1005600000F026FD0021416210BD426A1142F7D120
:1005700010BD2DE9F041046805460E46AC4214BF9B
:100580000027BDE8F081E0683043E060D4E9010174
:10059000826B0A438263017F082902D0092904D0B3
:1005A00009E0416A0A4206D002E0416A914302D161
:1005B00000F0FEFC47622468AC42E4D1BDE8F08163
:1005C000202181F31188C268002181F31188C16064
:1005D0001046704710B5202282F31188826B0024E8
:1005E00011438163027F082A02D0092A04D00AE05D
:1005F000426A114207D003E0426A32EA010102D1A5
:1006000000F0D6FC446200F0A4FD84F3118810BD14
:100610002DE9F0410E46202181F31188046805463A
:100620000027AC421BD0E0683043E060D4E9010110
:10063000826B11438163027F082A02D0092A04D009
:100640000AE0426A114207D003E0426A32EA01013D
:1006500002D100F0ADFC47622468AC42E3D100F067
:1006600078FD87F31188BDE8F0810022C168C2607F
:10067000084670472DE9F0410D0006464FF0000492
:1006800014BF0127BDE8F08107FA04F0284204D026
:10069000854356F8241020468847641C002DF3D16A
:1006A000BDE8F08170B5054652488469202080F38A
:1006B0001188A06B284005D10820656200F087FCF6
:1006C000A06B284041420840A16B8143A1630021F7
:1006D00081F3118870BD70B50546464884692020B5
:1006E00080F31188A06B284005D10820656200F0D6
:1006F0006EFCA06B2840A16B8143A163002181F3B4
:10070000118870BD70B505463A488469202080F391
:100710001188A06B35EA000003D00920656200F063
:1007200056FCA06BA843A063002080F311882846E4
:1007300070BD70B505462F488469202080F311886C
:10074000A06B4FF00006284007D041420840A16B43
:10075000814386F31188A16370BD41B108206562B1
:1007600000F077FC0028A4BFA06B2840EDDA86F3E8
:100770001188002070BD70B505461E488469202090
:1007800080F31188A06B4FF00006284005D0A16BC4
:10079000814386F31188A16370BD41B10820656271
:1007A00000F057FC0028A4BFA06B2840EFDA86F3C6
:1007B0001188002070BD70B505460E488469202060
:1007C00080F31188A06B4FF0000635EA00000AD0D4
:1007D00029B10920656200F03CFC002803DA86F3A9
:1007E0001188002070BDA06BA84386F31188A06318
:1007F000284670BDD00100205248514901600021B7
:100800008160C160103000F01FB900230360C0E9AF
:100810000213083AC1E90032103000F015B92DE991
:10082000F041050008BF474DC81D20F0070705F13E
:10083000080605F1100000F075F93068F8B10446BB
:100840004068B84217D307F1080188423CBF2068CE
:10085000306009D3E019216840F8081F6168C91B9E
:100860000839416030606760256000F089F904F163
:100870000800BDE8F081206826460028DFD100F09E
:100880007FF9296841B107F10800884700281CBF9B
:10089000E0E80257BDE8F0810020BDE8F08170B5C6
:1008A00050F8086CA0F1080406F1080506F11000E4
:1008B00000F038F92846854201D0AC4222D9296897
:1008C00009B1A1421ED921602C60616804F10800C1
:1008D0000A182068824205D14268114408316160DB
:1008E00000682060686805F108010144A14205D153
:1008F000616808440830686020682860BDE870407E
:1009000000F03EB92D68D6E770B50E46040008BF6A
:100910000C4C04F1100000F005F90020A168054618
:1009200031B10C4649686D1C084421680029F8D192
:10093000002E18BF306000F023F9284670BD00007B
:1009400077090008B0010020174820F00701174878
:100950000160174921F00701416070471349C01D2C
:1009600020F00702D1E900031B1A934232BF002096
:1009700002440A607047202181F311880B49C01D91
:1009800020F00702D1E90003A3EB000C00239445FB
:1009900032BF184602440A6083F311887047034847
:1009A00041680068081A70474716002000000020C0
:1009B0000040002000230360C0E901127047026874
:1009C0000A6001607047202282F3118802680A6081
:1009D0000160002080F311887047002A1ABF4FF091
:1009E000000C2023704710B483F3118804680C6056
:1009F0008CF3118801604468521E2144F4D110BC6C
:100A0000704710B5016800291CBF0A68026004D154
:100A1000826812B1406890470146084610BD10B583
:100A20000146202080F31188086800281CBF026856
:100A30000A6004D18A68002A1CBF486890470021D8
:100A400081F3118810BD00004060002181600060CA
:100A5000704770B5064684488569B06800285CD048
:100A60008168AA68914244D28260017F002938D00F
:100A7000042902D005293CD11CE0D0E90012116004
:100A8000D0E900124A60426A11460968914204D0D6
:100A9000D1F808C083686345F7D901604B684360AB
:100AA000486041680860406AAA688068816891422D
:100AB000DAD31EE0D0E900121160D0E900124A60DA
:100AC000426A11460968914204D0D1F808C083688F
:100AD0006345F7D901604A68426048604168086030
:100AE00007E0D0E900121160D0E900124A6000F07E
:100AF0005FFA34462468B44203D0A168A8688842EB
:100B0000F8D92C60616869606560696804200D60CF
:100B10006E62BDE8704000F05ABAB560E86BF060F4
:100B2000EE6370BD10B5202181F31188FFF791FFAE
:100B3000002080F3118810BD816800291CBF0020AF
:100B4000704749498A6982608A69D26BC260896943
:100B5000C86301207047202181F311888168002932
:100B600018BF002008D140498A6982608A69D26B27
:100B7000C2608969C8630120002181F31188704730
:100B800070B539488269202080F31188D46B002524
:100B9000E168D1632068A04208BFA56017D0106C3F
:100BA00049B10B688B421CBF9B68834288BF1846C3
:100BB000C9680029F5D190602068016821604C6007
:100BC000A060C16BE1600021C46300F074FA85F39A
:100BD0001188204670BD244810B58369DC6BE1683C
:100BE000D9632068A04204BF0020A06016D01A6C10
:100BF00049B1086888421CBF8068904288BF02469D
:100C0000C9680029F5D19A602068016821604C60AC
:100C1000A060C16BE160C46300F0CAF9204610BD5A
:100C200070B511488469202080F31188E06B00259D
:100C3000B8B10146C068E0630868884208BF8D60AB
:100C400008D002680A6051608860C26BCA60C163E4
:100C500000F0AEF9E06B0028EBD1206CA06000F052
:100C600078FA85F3118870BDD001002010B40024FB
:100C7000DDF804C0406041618161C0E90241114476
:100C800001610060C0E9073C10BC704770B50446C4
:100C9000C0686061A0610020A0602068A04214BF0D
:100CA0006FF0010570BD016821604C6000F080F9B3
:100CB00045622068A042F6D170BDD0E9053C82684B
:100CC000634504D1002A1CBF6FF00300704710B5C4
:100CD000521C82605A1C42611970D0E904128A4287
:100CE00024BFC16841610168814207D00A6802607F
:100CF0005060084600F05CF900214162002010BD00
:100D00002DE9F04104460D46202080F31188E16969
:100D100000291CBF204688470027A068002808BF7C
:100D20009E4E11D129001ED0B069446204606368F0
:100D300043606060426810600D2000F08AF900286E
:100D40000DDBA0680028EDD0401EA060A069411C0A
:100D5000A161226900788A429CBFE168A16187F3A2
:100D60001188BDE8F0814FF0FF30F8E72DE9F05F22
:100D700004460027D0F81C901D4692460E462020BF
:100D800080F31188DFF814824FEA070BB9F1000FE6
:100D90001CBF2046C847A068B8B921466DB1D8F835
:100DA0001800416201604A6842604860416808601A
:100DB00029460D2000F04DF920B18BF311883846FB
:100DC000BDE8F09FA0680028E7D0401EA060A069A1
:100DD000411CA161007806F8010B2169A0698142DC
:100DE0009CBFE068A0618BF311887F1CBAF1010AF7
:100DF0001CBF202080F31188C8D13846BDE8F09F81
:100E0000DDF800C0406041618161C0E90221114408
:100E100001610060C0E9073C704770B50446C068D6
:100E20006061A0612169081AA0602068A04214BF17
:100E30006FF0010570BD016821604C6000F0B8F8EA
:100E400045622068A042F6D170BD2DE9F04104460C
:100E500015468846202080F31188A06800270028C6
:100E600008BF4E4E18D1290010D0B069446204600A
:100E7000636843606060426810600D2000F0E9F82C
:100E8000002806DA87F31188BDE8F0814FF0FF30C3
:100E9000F8E7A0680028E6D0401EA0606069411C09
:100EA000616180F80080D4E9040188429CBFE06859
:100EB0006061E16900291CBF2046884787F31188DB
:100EC0000020BDE8F081D0E905328168934204D169
:100ED00000291CBF6FF00200704710B5491C8160EB
:100EE000511C816114780269914224BFC1688161FB
:100EF0000168814207D00A6802605060084600F02D
:100F000057F800214162204610BD2DE9F05F0446EC
:100F10000027D0F81CA01D4691460E46202080F3E5
:100F20001188DFF87880BB46A068B8B921466DB15A
:100F3000D8F81800416201604A6842604860416820
:100F4000086029460D2000F084F820B18BF3118849
:100F50003846BDE8F09FA0680028E7D0401EA0609A
:100F6000606916F8011B421C62610170D4E904013A
:100F700088429CBFE0686061BAF1000F1CBF204648
:100F8000D0478BF311887F1CB9F101091CBF2020C9
:100F900080F31188C8D13846BDE8F09FD001002009
:100FA000AF4800214060816000604061006170478F
:100FB00000210177AA49826809688B689342FBD2B5
:100FC00001604A6842604860416808607047A44B0D
:100FD0001A46996908771420C8771068D0F800C0BD
:100FE000C2F800C0CCF80420012298610277FFF714
:100FF00013B9202181F31188017F4FF0000C0029E3
:1010000004BF8CF311887047032904D0052918BF49
:101010000D290AD103E0416A8A68521C8A60D0E92E
:1010200000121160D0E900124A604FF0FF314162B6
:1010300080F81CC08A49826809688B689342FBD299
:1010400001604A684260486041688CF3118808601A
:101050007047F0B5824C054685B0A369481C4FF037
:1010600014074FF0010616D07E4A684600F099FA40
:10107000A16922460D77CF771068036813605A6024
:10108000A0610677FFF7C8F8039800281CBF6846E0
:1010900000F0A3FA0BE0724A1D77DF77106819465B
:1010A000036813605A60A0610677FFF7B5F8A0697E
:1010B000406A05B0F0BD30B4694C41628368A169F3
:1010C0000022D1F808C063459DBF027764491A46E3
:1010D0000A7784BF624A63460BD809688B689342DB
:1010E000FBD201604A68426048604168086030BCD9
:1010F00070471268D2F808C09C45FAD20A6053685B
:101100004B6051604A6811600122A061027730BCD7
:10111000FFF782B8DFF848C16046DCF818100268B3
:101120001368036058600120CCF818201077002065
:1011300008778A686046006883689342FBD8086035
:1011400042684A60416048680160DCF81800FFF7B7
:1011500063B8DFF80CC1DCF80000DCF81810826816
:101160008B689A4298BF70473D4A036813605A6083
:101170000122CCF8180002770020087738488A68E6
:10118000006883689342FBD8086042684A60416007
:1011900048680160DCF81800FFF73EB8DFF8C0C00F
:1011A0006046DCF81810026813680360586001207C
:1011B000CCF8182010771420C877002008778A68A8
:1011C0006046006883689342FBD2086043684B60C6
:1011D000416048680160DCF81800FFF71DB8F0B402
:1011E0001F4B00251846996900680126CA7FD0F870
:1011F00000C0C2B11A46C2F800C0CCF80420986101
:1012000006770D7710468A680068D0F808C09445C4
:10121000FAD8086042684A6041604868016098698D
:10122000F0BCFEF7F9BF0E4A0C46C2F800C0CCF87D
:101230000420986106771420C8770D7710468A68D5
:101240000068D0F808C09445FAD2086042684A6045
:1012500041604868016021469869F0BCFEF7DCBF38
:10126000D0010020F30F00082A4928A0896988616D
:10127000FEE708B5FFF73CF8FFF792FE00F088F9AB
:10128000FFF762FBFFF7B8FA4021234800F04CF863
:101290002049886101210177002181F3118862B61C
:1012A0001E4A8261AFF23F0300910122C0211C4817
:1012B00000F07EF808BD70B516488069C17F00292E
:1012C0001CBF491EC177016A491C0162154CE068C8
:1012D000401CE0602068A04208BF70BD8168491EC4
:1012E000816006BF0025202670BDC168C560026808
:1012F0005460026885F3118822600069884786F38C
:101300001188206881680029EFD070BD69646C6520
:1013100000000000D0010020F0010020E4310008AE
:1013200038020020F80200200222816002770022A9
:1013300042771423C377C0E90F218263026201213F
:1013400081779049826101614A69426148614169DE
:10135000086100F128018162091D0163C1627047C3
:1013600001442439DDF800C0C1600B60C168C1F8D8
:1013700004C0C36884491962022182600177002198
:1013800041771423C377C0E90F1281630162012200
:10139000827781617B4901614A69426148614169A3
:1013A000086100F128018162091D0163C162704773
:1013B00070B504464FF0200C8CF311882144243979
:1013C0000498E1600B60E16800254860E1686E48C0
:1013D00008620220A260207765771420E077C4E9D4
:1013E0000F52A56325620120A0776648A5612061A0
:1013F00041696161446160690021046104F1280070
:10140000A062001D2063E0622046FFF754FE85F3D2
:101410001188204670BD10B50146202080F3118848
:1014200058488069046C8268A24201D0914200D978
:1014300081600164FFF78DFE002080F31188204653
:1014400010BD10B50446202181F311880021FFF75B
:1014500032FE002181F31188204610BD202181F346
:101460001188417F41F004014177002080F3118809
:10147000704710B5202282F3118801460620FFF73D
:10148000E8FD002080F3118810BD10B5202181F304
:1014900011883E49C968411A1CBF0620FFF7D9FDD3
:1014A000002080F3118810BD10B5202080F3118832
:1014B00034480168806989688068814228BFFFF7E5
:1014C0006DFE002080F3118810BD70B52D498C6928
:1014D00004F128056062A06AA84207D0A06A0268E9
:1014E000A262FFF765FDA06AA842F7D1607F10F005
:1014F000030F05D1D4E904010861D4E90401416175
:10150000BDE870400E20FFF762BD70B5202181F369
:1015100011881C498C6904F128056062A06AA84200
:1015200007D0A06A0268A262FFF742FDA06AA84243
:10153000F7D1607F10F0030F05D1D4E904010861F1
:10154000D4E904014161BDE870400E20FFF73FBDC2
:1015500070B50446202080F31188207F0E2807D024
:101560000848A16A80690160A0620720FFF72FFD8B
:10157000002080F311882046656AFEF737FF284671
:1015800070BD0000D001002029020008F8020020F0
:1015900023484FF0FF314060816000210060C1604E
:1015A0007047DFF87CC0C0E90323DCF800209368B3
:1015B0008B4204D21268C91A93688B42FAD3026034
:1015C000536843605060436862451860816008BF9B
:1015D00070479068401A90607047114A01689142C4
:1015E00003D08A6883681A448A60D0E900121160C7
:1015F000D0E900124A600021C1607047084AD268F1
:10160000814207D9824228BF914201D90120704707
:10161000002070478242F9D28A42F9D2F6E70000F0
:10162000F802002000F079BF012101700021416023
:10163000704710B50446202080F311882046616071
:1016400000F072FF02202070002080F3118810BD8E
:1016500010B50446202080F31188204600F08EFF4C
:1016600001202070002080F3118810BD202282F319
:101670001188C068491E89B2C162002080F31188B8
:1016800070470322027000F092BF10B5202282F34F
:1016900011880322027000F08AFF002080F3118875
:1016A00010BD0422027000F082BF10B5202282F328
:1016B00011880422027000F07AFF002080F3118864
:1016C00010BD0221017000F009BF10B5202181F387
:1016D00011880221017000F001FF002080F31188C1
:1016E00010BD10B5044604202070204600F070FFA5
:1016F0000220207010BD000010B500F0FFFD00F0CA
:1017000024F9174800F09AFAFFF78CFF00F02CF844
:1017100000F090F8BDE81040FEF75CBD114A526839
:10172000814207D9824228BF914201D901207047E6
:10173000002070478242F9D28A42F9D2F6E7094B7B
:1017400059680A1858688A4204D9884228BF8242D8
:10175000F8D870478842F5D29042F3D37047000022
:101760003C310008001000E000F0A2BB0121017034
:1017700000214160704710B50446202080F3118895
:10178000616088882081204600F0A1FB0220207043
:10179000002080F3118810BD10B50446202080F38E
:1017A0001188204600F030FC01202070002080F3DA
:1017B000118810BD202282F3118801810069491E21
:1017C00089B2C162002080F31188704710B52023D0
:1017D00083F3118800F03CFC002080F3118810BDD9
:1017E00010B5202282F3118800F050FC002080F315
:1017F000118810BD4FF0FF333030FFF786BB4FF03C
:10180000FF330C30FFF7B2BA4FF0FF323030FFF742
:101810001CBB4FF0FF310C30FFF772BA3030FFF7CE
:1018200014BB0C30FFF76CBA3030FFF76EBB0C30D6
:10183000FFF79CBA00F066BC38B50446314820601A
:10184000201D60600120207215460B46102204F115
:10185000540104F10C000094FFF708FA2B46102203
:1018600004F1640104F130000094FFF7C9FA38BDB7
:1018700010B50446202080F31188204600F054FC67
:1018800002202072002080F3118810BD10B504469C
:10189000202080F31188204600F07FFC0120207278
:1018A00004F13000FFF7B9FA04F10C00FFF7EEF98C
:1018B000FFF74FFC002080F3118810BD70B504467F
:1018C00040690D4618B90421201DFEF752FE294635
:1018D00004F10C00FFF7F1F90028A8BF70BD8021CA
:1018E000201DBDE87040FEF744BE70B504463030A0
:1018F000FFF7E9FA051E03DA0821201DFEF739FE7D
:10190000284670BDFC3100081B494968816070475A
:10191000194949688268891A184A1268891A8160C7
:10192000C268914284BFC16070470269914288BF1A
:10193000114601617047124901601249416000215E
:101940008160C160491E0161704710B50B4C86B0C3
:1019500000200B49206000910A49CDE90110039055
:10196000401E04906846FFF7CFFF019968468847FC
:101970000298206006B010BD001000E008000020B2
:1019800009190008111900080FB42DE9F04F83B0B0
:1019900007460EAD4FF02D090D9810F8011B0D9064
:1019A000002902BF03B0BDE8F00F5DF814FB252944
:1019B00004D03868826838469047EDE701786C4675
:1019C00026464FF0000C2D2903D1401C4FF0010C8E
:1019D0000D9001784FF020082E2903D1401C4FF0C4
:1019E00030080D904FF0000B0D9911F8010B0D917F
:1019F000A0F13001092998BFC8B207D92A2803D01D
:101A000000212E2807D012E015F8040B0BEB8B01F8
:101A100000EB410BE8E70D9A12F8010B0D92A0F1D3
:101A20003002092A98BFD0B20ED92A280AD06C28D1
:101A300018BF4C280DD0A0F14102192A94BF0123F0
:101A4000002310E015F8040B01EB810100EB4101CC
:101A5000E1E7DDF834A001239AF800201AB110461E
:101A60000AF101020D92642839D00EDC552874D099
:101A700006DC442818BF492831D04F286FD010E029
:101A8000582868D063280CD10DE0732812D004DAEE
:101A9000692824D06F2804D161E075285DD07828AA
:101AA00059D0207004E015F8040B4FF02008207086
:101AB000641C87E055F8046B4FF02008002E08BF27
:101AC0005CA6002908BF47F6FF713446207800283D
:101AD00078D0491E0029A8BF641CF7DA72E055F8D7
:101AE000042B002A02DA04F8019B52420A21134611
:101AF00004F10B0A1046B2FBF1F201FB1200303088
:101B00003928C8BFC01D0AF8010DB3FBF1F3002B43
:101B1000F0D1A4EB0A0000F10B03012BD8BF012385
:101B2000AAF10101601E13F0010F03D011F8012F7B
:101B300000F8012F5A1009D091F801A080F801A0F7
:101B400011F802AF00F802AF521EF5D11C4439E083
:101B500003E004E0FFE7102202E00A2200E008228E
:101B600055F8040B04F10B03014600BFB0FBF2FA79
:101B700002FB1A0030303928C8BFC01D03F8010D20
:101B8000B1FBF2F150460029F0D1E01A00F10B0A46
:101B9000BAF1010FD8BF4FF0010A591E601E1AF0AA
:101BA000010F03D011F8012F00F8012F5FEA6A023C
:101BB00007D04B78437011F8023F00F8023F521EE5
:101BC000F7D15444A4EB060AABEB0A04002CB8BFCF
:101BD0000024BCF1000F08BF6442002C13DA3178F6
:101BE0002D2908BFB8F1300F06D13868761C8268FD
:101BF00038469047AAF1010A38684146826838465B
:101C00009047641CF8D1BAF1010A08D4386816F874
:101C1000011B826838469047BAF1010AF6D5002CBC
:101C20003FF4BAAE38684146826838469047641E31
:101C3000F8D1B1E6286E756C6C29000064490A6819
:101C400042F03F020A6063490A6842F03F020A60BC
:101C50000A6842F03F020A605F4942684A6082684F
:101C60008A60C268CA6002694A6142690A6282691E
:101C70004A6202680A605949026A4A60426A8A6096
:101C8000826ACA60C26A4A61026B0A62426B4A6235
:101C9000C2690A605249C26B4A60026C8A60426C37
:101CA000CA60826C4A61C26C0A62026D4A62826BCF
:101CB0000A604C49826D4A60C26D8A60026ECA60D9
:101CC000426E4A61826E0A62C26E4A62426D0A6068
:101CD0004549426F4A60826F8A60C26FCA60D0F81D
:101CE00080204A61D0F884200A62D0F888204A62B5
:101CF000026F0A603D49D0F890204A60D0F89420E5
:101D00008A60D0F89820CA60D0F89C204A61D0F848
:101D1000A0200A62D0F8A4204A62D0F88C000860A3
:101D200070472DE9F04F02F00305C2F38004C2F3BF
:101D3000C10CC2F34113C2F3C31700224FF00F08C6
:101D40004FF001094FF0030A11F0010F34D056078C
:101D50004FEAD66B07FA0BF608FA0BFB082A34BFDA
:101D6000D0F820E0D0F824E02EEA0B0B4BEA060670
:101D700034BF0662466209FA02F6D0F804B02BEAD4
:101D80000606264346605600D0F808B00AFA06F662
:101D90002BEA060B4BEA0C0BC0F808B0D0F80CB0DD
:101DA0002BEA060B4BEA030BC0F80CB0D0F800B0DE
:101DB0002BEA06062E430660490808BFBDE8F08FEF
:101DC00064009B00AD004FEA8C0C521CBCE7000085
:101DD0001C38024028380240000002400004024043
:101DE00000080240000C02400010024000140240B3
:101DF00070B5AF4C2069018A828902EA0105E94386
:101E0000018215F0020F03D06068016920468847FF
:101E100015F0040F03D0606881692046884715F0EB
:101E2000080F03D06068016A2046884715F0100F3C
:101E300003D06068816A2046884715F0010F03D0FF
:101E40006068816820468847BDE87040FEF7F6B9B3
:101E500070B5984C2069018A828902EA0105E9433C
:101E6000018215F0020F03D060680169204688479F
:101E700015F0040F03D0606881692046884715F08B
:101E8000080F03D06068016A2046884715F0100FDC
:101E900003D06068816A2046884715F0010F03D09F
:101EA0006068816820468847BDE87040FEF7C6B983
:101EB00010B57F48FFF75AFC7D497F48086101F162
:101EC0001400FFF753FC7B497C48086110BD2DE9E5
:101ED000F04104460078002501282CD020690580B7
:101EE00020698581206905822069456320698563B1
:101EF0002069C56320690564206945626168E068FE
:101F00000968B0FBF1F02169401E0885208921692C
:101F1000401E80B2C86260682169808D88806168D7
:101F200000200A7B02F00F02012A33D0022A08BFE8
:101F300002202FD030E05E48614F624EDFF888818A
:101F4000A0420ED1386840F002003860306840F09E
:101F500002003060356070211D20FEF7EDF9C4F8F5
:101F60000C805448A0420ED1386840F0040038601C
:101F7000306840F004003060356070211E20FEF7AC
:101F8000DBF9C4F80C80216946F6680008832169F2
:101F90008883B3E740F001000A7D02F00F02012AB6
:101FA00004D0022A08BF40F0200001D140F0100008
:101FB0000A7F02F00F02012A04D0022A08BF40F46F
:101FC000007001D140F4807091F8241001F00F01ED
:101FD000012904D0022908BF40F4005001D140F487
:101FE00080502169088421690120888260688068A6
:101FF000002818BF01202169888120690582216994
:1020000085200880BDE8F08170B50446007802287C
:1020100018BF70BD0020216908802169888121696D
:1020200008822348264DA04206D11D20FEF7A4F9C0
:10203000286820F0020028601E48A04218BF70BD2A
:102040001E20FEF799F9286820F00400286070BD72
:102050004FF0340C03690CEB810C43F80C20102377
:10206000426803EBC103D258002A08BF70470369D6
:102070009A894FF0020C0CFA01F1114218BF704717
:102080000A439A810069C943018270474FF0340CBA
:1020900003690CEB810C002243F80C200069828953
:1020A000022303FA01F122EA010181817047000055
:1020B000080300201C03002000040040000800402A
:1020C00024380240183802400048E8017F4801885F
:1020D00041F08001018070477D48018841F0800116
:1020E0000180704710B57B4800F077F8BDE81040DC
:1020F000FEF7A4B810B5784800F06FF8BDE81040BE
:10210000FEF79CB810B5754A00217248FFF794FBA2
:1021100070497348734A486700216F48FFF78CFB8A
:102120006D497148486710BD70B50C00054608BF81
:102130006E4C287A012817D16648A84208D16C480D
:10214000016841F480410160C0212520FEF7F4F8C8
:102150006148A84208D16748016841F40031016034
:10216000C0212620FEF7E8F85D4A63492268686FBF
:10217000B1FBF2F10181E18841F040010182218946
:1021800041F001018182A18842F22C121143818128
:10219000002101800188808870BD017A022918BF62
:1021A00070470022416F8A810A828A8249498142AE
:1021B00007D14F48016821F4804101602520FEF7D6
:1021C000DBB84549814218BF70474A48016821F48D
:1021D000003101602620FEF7CFB82DE9F047456FAA
:1021E0000646B5F80C902C88B5F804A014F00F0F33
:1021F0004FF020074FF000081AD0002114F0080F0C
:1022000018BF802114F0010F18BF41F0200114F015
:10221000020F18BF41F0400114F0040F18BF41F441
:10222000807187F31188301DFEF7A3F988F31188B8
:1022300014F4807F0CD087F311884FF40071301DA7
:10224000FEF797F988F31188288820F48070288099
:1022500014F0200F08D087F311880AF0FF013046F0
:10226000FFF72CFB88F3118819F0800F18BF14F0CA
:10227000800F14D087F3118806F13000FEF723FE9B
:102280000028A8BFA88008DA0821301DFEF771F9E0
:1022900029F0800040F04000A88188F3118814F0F4
:1022A000400F08BFBDE8F08787F311881021301D6B
:1022B000FEF75FF988F3118829F04000A88128888B
:1022C00020F040002880BDE8F08700000C38014075
:1022D0000C44004030030020A8030020CD2000085B
:1022E00000380140D9200008004400401C3200089A
:1022F00020380240243802400048E8016B49086851
:102300000860002008606A490A680A600860091FBE
:102310000A6842F001020A6008604FF0E02147F6C7
:10232000FF424A618861072008616248016841F004
:10233000807101606048016841F0010101605F48FF
:10234000016841F0805101605D48016841F480718D
:1023500001605C48016801F44031B1F5803F07D06D
:10236000016841F400010160016821F4000101608D
:10237000016841F480710160016811F4007FFBD0B5
:10238000016811F4800F18BF7047016841F4803173
:102390000160016841F480010160704747494FF0D6
:1023A00080500860464B586810F0100FFBD14FF476
:1023B00000601860586810F0100FFBD1424A0020EE
:1023C0001060101F016821F4604141F42041016058
:1023D0003C49800508603D484FF4807CC0F800C04F
:1023E000D0F800C01CF4007FFAD0D0F800C04CF048
:1023F000010CC0F800C000BFD0F800C01CF0020FF4
:10240000FAD0D1F800C04CF0010CC1F800C000BFF8
:10241000D1F800C01CF0020FFAD0D1F800C01CF4B3
:10242000807F11D1D3F800C04CF4807CC3F800C089
:10243000D1F800C04CF4807CC1F800C0D3F800C0D3
:102440002CF4807CC3F800C00B6813F4007FFBD031
:10245000136843F408031360036843F08073036058
:10246000036813F0007FFBD00368036010681060FE
:10247000086840F480300860154804210160072195
:102480000160106840F0030010600C20116830EA11
:102490000101FBD10F48016841F0010101600E48C4
:1024A000016841F0010101607047000010380240EE
:1024B00018380240FCED00E0001000E02438024033
:1024C00000700040343802400838024000380240B2
:1024D000003C0240203802402C380240C2680021F3
:1024E0001180C2681182C06881817047414810B56F
:1024F000C268002111820278042A07D102220270E8
:10250000C2681180C2681182C268918141684968BD
:102510008847BDE81040FDF791BE36494FF0804036
:10252000C8600846FFF780B870B5044600780025FB
:10253000012804BF2F48A04210D12F48016841F064
:10254000010101602D48016841F001010160056051
:1025500070211C20FDF7F0FE2948A060D4E901108D
:102560000968B0FBF1F0E168401E0D80E2680821C7
:102570009180E1680885E068858170BD0178022955
:1025800018BF70470021C2681180C2689181C2687B
:1025900011821849814218BF704710B51C20FDF701
:1025A000EBFE1548016821F00101016010BDC26811
:1025B000491ED162C26801219182C36800225A6219
:1025C000C3681A82C2689181C06805210180704782
:1025D000C268491ED162C26801219182C26800218D
:1025E0001182C2680D211180C068018A11F0010FAB
:1025F000FBD07047200400202438024018380240E5
:102600000048E80170B5202080F31188FB4D0024BC
:10261000286820B132214162FEF7CAFC2C6084F3A5
:10262000118870BDF64810B5417A41291CBF0020C1
:1026300010BD00F12601F348FFF7A6F9F2A1F14819
:10264000FFF7A2F9EE49EF48FFF79EF9EEA1ED483A
:10265000FFF79AF9012010BD82B0DFF8C0834FF474
:10266000FA7000250090D8F81810E8A0DFF88CA3C5
:102670002F462E460124AB464FF02009C1F8180022
:1026800089F31188D8F81800CAF800000220FEF774
:102690009EFCD8F81800406A8BF3118801280FD0EF
:1026A000022813D0322841D0012FE9D1012EE7D8DA
:1026B0000226052DE4D2DFE805F03C7394B4D30084
:1026C0000127701CC6B200253C46EFE7D4484FF402
:1026D00080610180C1140180811401804900018062
:1026E000012F08D0CFA1C748FFF74EF9C448417A5F
:1026F000412916D104E0D2A1C248FFF745F9F5E718
:1027000000F12601BF48FFF73FF9BFA1BD48FFF721
:102710003BF9BB49BB48FFF737F9BBA1B948FFF705
:1027200033F900273E463D460124A9E7012FA7D1F2
:10273000BEE7012C1AD0142CA2D800BF04EB8402EF
:10274000C7A1B048FFF720F9D1494FF48060088055
:10275000D0480099FEF7A9FF601CC4B2152C8FD198
:10276000A9A1A848FFF710F9012538E0CAA1A5489A
:10277000FFF70AF9A248417A4129DFD100F1260189
:10278000A048FFF701F9A0A19E48FFF7FDF89C497A
:102790009C48FFF7F9F89CA19A48FFF7F5F8CDE7B8
:1027A0000A2C3FF66DAF9E484FF480610180B84916
:1027B000C014088004EB84004200BDA19148FFF7DB
:1027C000E3F8B4480099FEF770FF601CC4B20B2C0C
:1027D0007FF456AF8CA18B48FFF7D6F80225012471
:1027E0004EE70A2C3FF64CAF8D484FF40061018054
:1027F000A7498014088004EB84004200B4A18148FA
:10280000FFF7C2F8A3480099FEF74FFF601CC4B25F
:102810000B2C7FF435AF7CA17A48FFF7B5F8032580
:10282000DDE7142C3FF62CAF7D484FF4805101803A
:1028300048009749088004EB8402AEA17148FFF775
:10284000A3F894480099FEF730FF601CC4B2152C21
:102850007FF416AF6CA16B48FFF796F80425BEE72E
:102860006F494FF400500880AAA16648FFF78CF822
:102870006348417A412910D100F126016148FFF7F0
:1028800083F861A15F48FFF77FF85D495D48FFF776
:102890007BF85DA15B48FFF777F800273E463D4691
:1028A000EEE65E49ADF5487DA0A08969544DA24E83
:1028B00000270DF52F7888614FF46170FEF7D9FD80
:1028C0004FF0FF334FF42F72694606F10C00FEF70C
:1028D0004DFA9AA1684600F027FB5FEA000955D03F
:1028E00098A100F021FB00283AD0A0EB0900C4B267
:1028F000642C88BF642422464946AFA800F058FBE8
:102900002146AFA800F086FA05F10B028EA18A4895
:10291000FFF73AF805F118028FA18748FFF734F85E
:1029200005F1260290A18448FFF72EF805F109026F
:1029300090A18148FFF728F8314A92A17E48FFF71D
:1029400023F808F80470AFA97B48FFF71DF84FF093
:10295000FF3302222CA106F13000FEF7D6FAABE7D6
:102960004FF0FF33022228A106F13000FEF7CDFA26
:1029700087A17148FFF708F84FF0FF334FF42F722B
:10298000694606F13000FEF7C0FA95E78BA16A4868
:10299000FEF7FAFF90E7F0B59BB0074690A100F074
:1029A00033FB2026154C0025C8B18FA1384600F016
:1029B0002BFB08B38EA1384600F026FBE8B16C2251
:1029C0008D49684600F0C2FA69460E48FEF7DCFF02
:1029D0008A48016881F0800101601BB0F0BD86F378
:1029E0001188206820B101214162FEF7E1FA2560DB
:1029F00085F311881BB0F0BD02E10DE10C00002051
:102A0000100A0020300300200D0A00004F6470619E
:102A10006C5F766C616B6E6F00000000D00100206F
:102A20001A0402404F6470616C206E6562796C20FC
:102A3000616B7469766F76616E2E0D0A000000007E
:102A40000D0A4F6470616C207A727573656E207523
:102A50007A69766174656C656D2E0D0A0000000060
:102A600028312F34290956656E74696C206F74659E
:102A70007672656E202D3E206E6166756B6F766195
:102A80006E692062616C6F6E7520256425250D00CE
:102A900018040240200400205679706F7573746525
:102AA0006E69207A6168616A656E6F210D0A0000A7
:102AB00028322F34290950726570616C6F76616E0F
:102AC00069206C6973752E2E2E20256425250D0036
:102AD00028332F3429095A617461766F76616E69E3
:102AE0002062616C6F6E752E2E2E20256425250DBB
:102AF0000000000028342F3429094F74657669726C
:102B0000616E692076696B612E2E2E202564252545
:102B10000D0000005679706F757374656E692075CD
:102B20006B6F6E63656E6F210D0A00004750535F37
:102B30004E4D454100000000A8030020244750529C
:102B40004D4300002A0000004C617469747564658F
:102B50003A2025730D0A00004C6F6E676974756426
:102B6000653A2025730D0A00446174756D3A20257D
:102B7000730D0A005374617475733A2025730D0A3E
:102B8000000000004361733A2025730D0A00000025
:102B90004E656E616C657A656E20756B6F6E636FE6
:102BA00076616369207A6E616B204E4D4541207AD3
:102BB0007072617679202A0D0A0000004E656E6100
:102BC0006C657A656E207A61636174656B2047502D
:102BD000524D43207A70726176790D0A0000000030
:102BE0006F6470616C0000007A7275730000000001
:102BF00068656C70000000003C320008140402405C
:102C000086F31188206800283FF4F2AE0221416269
:102C1000FEF7CEF92560EBE61BB06C49BDE8F0404D
:102C20006B48FEF7B1BEA6B00025FEF765FDFEF7C6
:102C300020FB00216648FEF71BFE664C40F2823204
:102C40004FF400712046FFF76CF840F282322115F4
:102C50002046FFF766F860496048FEF709FE40F23B
:102C6000823204212046FFF75CF840F282320821CC
:102C70002046FFF756F85A4E012280213046FFF7D2
:102C800050F858495848FEF776FD4FF481724021BC
:102C90003046FFF746F842F2107200215248FEF724
:102CA00095FD012291023046FFF73BF820154F4C6D
:102CB0002080410001223046FFF733F8E0142080E5
:102CC000410001223046FFF72CF8A014208041007B
:102CD00001223046FFF725F84FF400502080444988
:102CE0004448FEF7A6FC0024434B40224FF4966173
:102CF00042480094FEF75CFB414B40224FF4987130
:102D000040480094FEF754FB30493148FEF73CFE42
:102D1000DFF8BC903C4E4FF0010A4FF0200806AFA0
:102D20004FF0FF33012201A909F10C00FEF71EF854
:102D30009DF804000D2801D00A2D41D300250DF186
:102D4000180BAFF26411584600F05EF9E8B1AFF22B
:102D50006811584600F058F908B3AFF26C115846A4
:102D600000F052F938B36C2228490AA800F0EEF8B6
:102D70000AA91748FEF708FE2548016881F080017E
:102D8000C0F800108DF81840CAE788F31188306841
:102D900070B1C0F824A0FEF70BF9346008E088F3A6
:102DA0001188306820B102214162FEF701F93460D8
:102DB00084F31188E6E705490548FEF7E5FDE1E7FC
:102DC00079194C707855681CC5B2A9E7100000202D
:102DD000300300200000024030320008A803002029
:102DE000000402407C0100201C0300201A04024061
:102DF0002832000820040020A328000860050020D5
:102E000059260008300400200C0000203C32000845
:102E1000140402402DE9F04F002214461646904655
:102E2000154613461746002998BFBDE8F08FDFF816
:102E3000F4C04FF03A094FF02E0A52E0012B0CD0AB
:102E4000022B21D0032B18BF042B24D0052B18BF35
:102E5000062B29D0092B44D131E010F802B0BBF188
:102E60002E0F08BF012756D047BB022C18BF052CD8
:102E700003D10CF80490641CE4B210F802B00CF812
:102E800004B0641CE4B22CE000EB020B1BF801BCA4
:102E90008CF809B025E00CEB060E10F802B0761C99
:102EA0008EF80BB0F6B21CE00CEB080E10F802B076
:102EB00008F101088EF818B008F0FF0811E0022DA3
:102EC00018BF052D05D10CEB050B6D1C8BF826A04A
:102ED000EDB20CEB050E10F802B06D1C8EF826B0AA
:102EE000EDB210F802B0BBF12C0F04BF5B1CDBB2DB
:102EF000092B10D900200CEB06010CF80400887295
:102F00000CEB0801C8750CEB050181F825008CF865
:102F10000A00BDE8F08F521CD2B291428ED8BDE8B3
:102F2000F08F0000100A002030B505460B462A46F7
:102F300013F8014B12F8010B08B1A042F8D01CB1F4
:102F4000002802D06D1CF1E7284630BD10B5203AAC
:102F5000C0F00B80B1E81850203AA0E81850B1E852
:102F60001850A0E81850BFF4F5AF5FEA027C24BF08
:102F7000B1E81850A0E8185044BF18C918C0BDE8FF
:102F800010405FEA827C24BF51F8043B40F8043BC8
:102F900008BF7047D20728BF31F8023B48BF11F87D
:102FA000012B28BF20F8023B48BF00F8012B7047D7
:102FB00010B5044610F0030F08BF11F0030F40F0E6
:102FC00015804FF0013E121FC0F20E8051F8043BF5
:102FD000A3EB0E0C2CEA030C1CEACE1C08BF40F835
:102FE000043BF0D0A1F1040102F10402521E08DBFF
:102FF00011F8013B002B00F8013BF7D1114600F01E
:1030000046F8204610BD00004FF0013C50F8042B5C
:1030100051F8043B9A4221D1A2EB0C03934313EAEB
:10302000CC1317D150F8042B51F8043B9A4215D118
:10303000A2EB0C03934313EACC130BD150F8042BEF
:1030400051F8043B9A4209D1A2EB0C03934313EAD3
:10305000CC13DBD04FF00000704700BFD01A01BA8C
:10306000B1FA81F101F0180122FA01F0CB40C1F16F
:103070002001DBB2C0B2C01A2CFA01F3D11A91437D
:1030800011EAC311E6D170477047704770474FF09F
:1030900000020429C0F0128010F0030C00F01B8025
:1030A000CCF1040CBCF1020F18BF00F8012BA8BF33
:1030B00020F8022BA1EB0C0100F00DB85FEAC17CF7
:1030C00024BF00F8012B00F8012B48BF00F8012BAA
:1030D00070474FF0000200B51346944696462039DB
:1030E00022BFA0E80C50A0E80C50B1F12001BFF4C1
:1030F000F7AF090728BFA0E80C5048BF0CC05DF827
:1031000004EB890028BF40F8042B08BF704748BF74
:1031100020F8022B11F0804F18BF00F8012B7047E8
:103120000446AFF300802046FDF74CF80149182013
:10313000ABBEFEE72600020070470000000000A8BA
:1031400000000000000000FC54555565FFFF000022
:10315000000000000000000080520000000000009D
:10316000F0F30000050555553FFF0000000000008A
:10317000000000000000000000000000000000F05F
:1031800055555505FFFF000000000000000000003D
:1031900000000000000000000000000055555555DB
:1031A000FFFF000000000000000000000000000021
:1031B000000000000000000055555555FFFF0000BD
:1031C00000000000000000000000000000000000FF
:1031D0000F00000050555555FFFF00000000000093
:1031E000000000006D61696E001642110404480879
:1031F0000C101418001C1D1E1F200000F5170008DD
:10320000FF17000809180008131800081D18000807
:1032100023180008291800082F180008802500002E
:103220000000004000000000E80300000526000840
:103230008025000000000040000000004E65706C1A
:1032400061746E79207072696B617A210D0A093C94
:103250006F6470616C3E2070726F207A6168616A81
:10326000656E692073656B76656E63650A0D093C52
:103270007A7275733E2070726F207A727573656E04
:1032800069207679706F757374656E690A0D093CF3
:1032900068656C703E2070726F206E61706F76652D
:1032A00064750D0A00000000C8320008000000200C
:1032B000AC01000030010008B0330008AC01002070
:1032C000941400008C01000801100F2F0D0A0D0A44
:1032D0002A200278560D0A5669746120766173209F
:1032E0004175746F6D617469636B79205679706F85
:1032F0007573746563204D6574656F62616C6F6E84
:103300007520312E310D0A5A61706F6A656E692021
:103310007679766F64753A0D0A094750494F423104
:1033200030202D2076656E74696C131A31137C6C15
:103330006973101A32101D7A617461274B69205528
:10334000791C1A331C2E6F746576721C1D6B727992
:10335000741B28085072696B617A796418083C6F95
:103360006470616C3E3F3B68617F1C73656B471BFB
:1033700063658849AC180B6E690A0D093C7A727551
:103380007326190649A4A91C180868656C703E20AC
:103390006EC108092F766564610D0A2A2002150D99
:1033A0000A0D0A23102763204E72016908011400D8
:04000005080000F5FA
:00000001FF
